:020000020000FC
:100000001FC0F3C027C127C131C12BC128C128C1DE
:1000100029C122C122C122C127C127C124C127C1B0
:0200200027C1F6
:10004000F89411E00EE51EBF0DBF00E811E006BDFB
:1000500016BD00E00BBB0FEF0ABB03E008BB00E0DE
:1000600007BB01E005BF00E000B900E000BF03E00E
:1000700003BF00E00CBF00E00CBF00E003BD04E0E4
:100080000FBD01E00EBD00E002BD00E00DBD00E0CF
:100090000CBD00E00BBD00E00ABD00E009BD00E0C2
:1000A00008BD00E005BD00E005BD00E007B900E0C7
:1000B00006B900E003B900E001B900E808B9A89565
:1000C00004B7077F04BF01B5006101BD0EE001BDAB
:1000D00000E70ABF07E008BF07E20BB900E002BB78
:1000E00000E000BD00E40BBF00E009BF00E00CB978
:1000F00007E1102E00E7002E75EA0CEC202E90E0B0
:10010000789442E30AEFE8D00AEFE6D00AEFE4D0B1
:100110000AEFE2D0F894112D002D78943CE120E212
:10012000201B310B30F44A9569F780E0CBD0009565
:10013000BAD070E0B1E0A4EF889427FC0894221CA8
:100140002BBA00E5C9D01197B9F780E0BBD000FF0A
:1001500001C002C0926001C09D7F91FF01C003C039
:10016000F1E0E2E502C0F2E0E0EF7894A895F894BF
:10017000112D002D789430E02BE07BD01F1719F45F
:100180000E1709F42DC091FF01C015C00E1B1F0BE7
:1001900048F4889427FC0894221C2BBA31970AE073
:1001A0009BD022C0889420FC089427942BBA0AE0A4
:1001B00093D0319619C00E1B1F0B48F4889420FC75
:1001C000089427942BBA0AE087D031970DC0889401
:1001D00027FC0894221C2BBA31960AE07DD004C07B
:1001E00000E00BBB0AE078D0C1CFFFB60F931F939E
:1001F0002F933F9306B302FD23C00CB51DB537E026
:1002000020ED201B310B00F537E220E1201B310BE4
:10021000D8F03FE020EA201B310B28F01FE000EA75
:10022000112E002E11C03FE120E4201B310B28F4D9
:100230001FE100E4112E002E07C0112E002E04C075
:1002400010E000E01DBD0CBD3F912F911F910F915B
:10025000FFBE189518951895189518951895189526
:100260001895189518951895189518951895189526
:1002700018954F935F936F934427552760E1000FC4
:10028000111F441F551F4217530718F00395421BB7
:10029000530B6A95A1F75F934F932F913F916F9105
:1002A0005F914F9108951F93E199FECF10E01CBB21
:1002B00010E01FBB8EBB0DBB753A11F4E29AE19AB8
:1002C0001F9108951F93E199FECF10E01FBB8EBBD5
:1002D000E09A0DB31F9108951F9314E600001A953C
:0C02E000E9F7A8950A95C9F71F91089549
:00000001FF
